S123E0007EED71BDECF7FEFFC4A60A815526040EBDF158BDE068FCFFC0F3FFC28F350E4F66
S123E0205FDD3ADD3FDD41BDE0AB7F00197F00187F001DBDE105BDE0BBBDE05BBDEE471A1A
S123E04083000026D1DE0ADF2FBDE1277D001926C520D7DE2F6F00DF0A20BBBDE3BA8120D4
S123E0602605BDE3C320F439CEE06E7EE11C0D0A0D0A424153494331312076312E35330DCE
S123E0800A436F7079726967687420313938352D313938392062790D0A476F72646F6E201F
S123E0A0446F7567686D616E0D0A00CEE0B17EE11C0D0A52454144590D0A00C64FDE49BD9C
S123E0C0FED5810D272B5D272881082610C14F2720098620BDFEB88608BDFEB85C8103269E
S123E0E0067C001C7EF26C812025D4A700085A26CE860DA700DE49DF003981612506817A8A
S123E100220284DF39CEE10A20120D0A23008D00CEE1198D077F001E390A0D00A60027066D
S123E120BDFEB80820F639DE4BDF028D3F241936BDE3BA810D322609BDEB9EDE0A08DF2D3D
S123E140397F00198D6E2010BDE3BA810D27F186019719CC000020ECBDE1E27D0019270370
S123E1607EF22BBDEB77DE0A08DF2D39183C4F36361830DE00A6008D422410A6008D3C253A
S123E180110D18EC0026048612200D31311838DF00398D072AE586017EEA9518EC0005056B
S123E1A018E3000518ED00E60008C0304F18E30018ED0039BDE3CB4F7EE3CE8130250681AA
S123E1C03922020D390C398141250E815A230881612506817A22020D390C398DEA240139CC
S123E1E020D9BDE3BA810D274F7F001ABDE371CEE246BDE39C251308A60026FBC6043A6D70
S123E2000026EF8602CEE4132004A601EE02BDE3CE810C2707810A2703BDE371AD00BDE3A1
S123E22071BDE3C1813A2607867ABDE3CE20B3810D270586027EEA95867DBDE3CEDC0293BE
S123E2404BDE4BE7023944415441000CE3F34C45540001E41352454144000DEA55524553F9
S123E260544F5245000EE3F2474F535542000FE3E9474F544F0012E3E94F4E54494D45003F
S123E28025E8D04F4E4952510026E8D04F4E504143430028E8F04F4E0013E8825245545528
S123E2A0524E0014E3F249460015E904494E5055540016EA3D5052494E540003E9D53F00E6
S123E2C003E9D5464F520004E96D4E4558540005E9C853544F500017E3F2454E445748009B
S123E2E01AE3F2454E440018E3F252454D000AE3F354524F4E0006E3F254524F46460007FD
S123E300E3F25748494C450019EA88504F4B450008E7F744494D0009EA55454550001BE80C
S123E32010504F525441001CE40F504F525442001DE40F504F525443001EE40F504F5254BF
S123E34044001FE40F494E425954450023EA8054494D450024EA90524554490027E3F250BE
S123E360414343000BEA90534C4545500029E3F2003CDE005FA600812026045C0820F65D15
S123E38026023839DF00DE02C101270C867FA70008E70008DF023839C67E20F5DC00373695
S123E3A0A60027128D1BBDE0FAA10027063233DD000C390820EA32330D393CDE00A6003831
S123E3C0398DF73CDE0008DF0038398D01173C3736DE02A70008DF02DC4BC300801A930233
S123E3E0323322E586147EEA9586A88DE1BDE16C20D939DE023C86008DD4C6028DBC810D9C
S123E40027078DCA8DBD5C20F38DC338E70039C6012004BDE554168DA8813D270586037EF5
S123E420EA9586798DA817183C361830CEE548BDE4F424028D98BDE3BA81282622BDE3C3B3
S123E4408610BDE3CE18A600BDE427BDE3C18129270586047EEA958611BDE3CE7EE48EBDBE
S123E460E1BB25088124270481222605BDE6692009BDE7644D2603BDE55418E600C10026A3
S123E4800318A70018A100270586057EEA95BDE3BA810D2740813A273C81202738812C2708
S123E4A034813B27308129272C18A60081012618BDE4DF2518BDE4EA25137D001A2705BD96
S123E4C0E4EF20098600200586137EEA954D260986067EEA9531183839BDE3CE7EE42CCE72
S123E4E0E50ABDE4F42502860039CEE51D20F3CEE53220EEBDE39C250D08A60026FB08088B
S123E500A60026F00C39A6010D392B00402D00412A00502F00515C00525E0060002E414E0D
S123E520442E00202E4F522E00212E454F522E0022003C3D00323E3D00333C3E00353C007F
S123E540303E00313D0034002D00724000704E4F54007100183C4F363636361830BDE3BAD9
S123E560BDE1C7250586077EEA95BDE0FA18A700BDE3C3BDE3BABDE1DB2409BDE0FA18A76F
S123E58001BDE3C3BDE5DD18A703BDE5EB1A83FFFF260618A603BDE623373618A603BDE329
S123E5A0CE3233BDE3CB18A6038510271EBDE3C38610BDE3CE8601BDE427BDE3C181292736
S123E5C005860E7EEA958611BDE3CE860118E603C50227028602313131311838398684360F
S123E5E0BDE3BA81283226028B1039DE086D00272EA1002612E60118E100260BE60218E173
S123E6000126048F930839E600C5102704C6052006C1842605C6053A20D386087EEA95CCD2
S123E620FFFF39DE0A3CA7000818E600E7000818E601E700088D186F00DF0A9C102304869B
S123E640092023323393083736BDF2DB32333985102704C602200681842609C6026F0008B4
S123E6605A26FA3986087EEA95BDE3BADE003C81242608BDE3C3BDE6CC2003BDE69E36861F
S123E680A4BDE3CE32BDE3CBDC0030A30017BDE3CE38A600BDE3CE085A26F7860139183CB4
S123E6A04F36361830DE00A600BDE1BB25048602202CA600BDE1BB2409BDE19B2AF4860A66
S123E6C0201CDF0018EC003131183839183C4F36361830DE00A600BDE71E250D860B7D004F
S123E6E01D27037EEAEC7EEA95A600BDE71E24D218EC0005252405252105251E05251B18DE
S123E700ED00A600BDE0FA1608C030C1092302C0074F18E30018ED0020CF860C20C0BDE1B9
S123E720BB240139BDE0FA81412506814622020D390C39C60286A2BDE3CEDE023C4FBDE359
S123E740CEBDE3C1BDE3CEBDE3C18122270F810D2605860D7EEA95BDE3CE5C20EABDE3CE53
S123E76038E70039CEE785BDE39C250E08A60026FBC6043A6D0026EF4F398636BDE3CEA6E7
S123E78001EE026E00464449560001E7FE434852240002E81C4142530004E81C524E44003E
S123E7A005E81C53474E0006E81C5441420007E81C4144430003E81C43414C4C0008E81C81
S123E7C05045454B0009E81C454550000AE81C484558320012E81C484558000BE81C504F5B
S123E7E05254000CE86554494D450011E87C504143430013E87C00DE0209DF02A600183C20
S123E800C60137371830C602BDE82B3232183839DE0209DF02A6008D037EE417183CC6015E
S123E82037C60118308D0432183839BDE3CEBDE3BA81282705860E7EEA95BDE3C38610BD5E
S123E840E3CE18A600180837BDE427335A2707BDEA2A24E120ECBDE3BA812926D8BDE3C324
S123E86086117EE3CEBDE3C1BDE0FA81412405862F7EEA95814522F780418B0CBDE3CE860E
S123E88001398601BDE427BDE371CEE271BDE39C240D8612BDE3CEBDE371BDE3E92018CEA6
S123E8A0E268BDE39C2505860F7EEA95860FBDE3CEBDE371BDE3E9BDE371BDEA2A25013934
S123E8C0BDE37186A8BDE3CEBDE16CBDE3CB20E78601BDE427BDE371BDEA2A250586157E97
S123E8E0EA95BDE37186A8BDE3CEBDE16C7EE3CB8D0220DC8601BDE427BDE371BDEA2A24D2
S123E900DC7EE3717C001A8601BDE427BDE371CEE963BDE39C250586107EEA958638BDE3DE
S123E920CEBDE371BDE3BABDE1BB242786A8BDE3CEBDE16CBDE3CBBDE371CEE968BDE39C79
S123E9402501398639BDE3CEBDE371BDE3BABDE1BB250586127EEA9586A8BDE3CEBDE16CFE
S123E9607EE3CB5448454E00454C534500BDE5548101270586037EEA95BDE3C1813D26F4AC
S123E9808679BDE3CE8601BDE427BDE371CEE9C0BDE39C250586117EEA958637BDE3CEBD4D
S123E9A0E3718601BDE427BDE371CEE9C3BDE39C250139863ABDE3CEBDE37186017EE4273B
S123E9C0544F005354455000BDE5548101270586027EEA9539BDE3BA8123260D8678BDE323
S123E9E0CEBDE3C3BDE371201BBDE371BDE3BA810D2704813A260139BDE3BA81222605BD72
S123EA00E73320058601BDE427BDE371BDE3BA810D27E4813A27E08D1125CE813B2705869F
S123EA20167EEA95867B8D0D20BFBDE3BA812C27020C39867CBDE3CEBDE3C30D398D21BD4C
S123EA40E371BDE3BA8122260CBDE7338DDC250586157EEA95BDE554BDE3718DCD25F63978
S123EA60BDE3BA81232701398678BDE3CEBDE3C3BDE3718601BDE427BDE3718DAD24D1398B
S123EA808DDEBDE3717EE5547C001A86007EE427C6017EE4179718BDE10EDE49A600810DA4
S123EAA02706BDFEB80820F4BDE110DE0009099C49230EDF00DE49862ABDFEB8089C0026EF
S123EAC0F8CEEADFBDE11CBDE1108D078601971C7EE053CEEAE3BDE11CD6184F7EEB175E4C
S123EAE05E5E004552524F52202320009718BDEAD3CEEB0BBDE11CDC29BDEB17BDE11086CA
S123EB0001971C7EE016425245414B20494E204C494E45202320001A830000260586307E06
S123EB20FEB8183C3736CC271037365F37183018EC032A0D4353C3000118ED03862DBDFEFE
S123EB40B818EC03CDEE010218ED038F1A8300002605186D00270B178B30C60118E700BDC9
S123EB60FEB818EC01CE000A02CDEF0126D3C605183A18351838398601971CDE4BEC001AEA
S123EB80930C230ABDEC66DE4BEC00DD0C398D56EC003CDE4B1AA30038266A7EEC8337364C
S123EBA018301A930C23078601971C3233398D36EC00CDA30026F0E6028D0DDC0CCDA3003F
S123EBC026E58D31DD0C20DF183C3C1838183A189C06240A18A600A70008180820F1DF06E3
S123EBE0BDECC6183839DE041AA300230737E6023A3320F439DE049C062709EC0037E602B8
S123EC003A3320F3393CDE4BE602383C8D03382040183C3CDE0A3A9C0E222BBDECA0DE0678
S123EC203C3A3C183018EC00DD0618EC02CDA3042519CDEE02A60009CDEF02CDEE00A700AB
S123EC4009CDEF0020E486097EEA953838381838393CDE4BE6023818DE4B18A6001808A7DF
S123EC6000085A26F539DE4BE602DE0A3A9C0E220DBDECA0DE063A8FDE06DD0620D386098F
S123EC807EEA95E6023CDE4BE00238260220C22A08503CBDEC113820B83CBDEBC83820B1C5
S123ECA0183C37DE0A18DE0A3ADC0ADF0A9308270FDD6C18A600A7000918098D322AF40846
S123ECC0DF0833183839183C3718DE0886FF50D3088FDC0A9308DF08DD6C270D18A600A77B
S123ECE0000818088D092AF409DF0A33183839DC6C830001DD6C39FEFFC0DF08DF0ADF04C8
S123ED00DF068FF3FFC2830251DD10DD0EC30001DD49C30050DD4BC30080DD4DC3001EDDC9
S123ED204FDD51C3003CDD53DD55C30050DD57DD59C30010DD5BDD5DC30010DD5FDE046FCF
S123ED4000089C0E23F9FEFFC4A60A81552603BDF3A7CC0000DD0CDD29BDF2837F001B860D
S123ED6001971CFEFFCEA7007F0037DE0A08DF2D39FCFFC8DD6144444444B7103DDE6186A4
S123ED8093A7398603A724FCFFC0F3FFC28F35CE00C418CEEDFAC614867EA700081AEF0080
S123EDA008085A26F5CE00F7CCED71ED01ED04ED07CE00A418CEFFA0C62018A600A70008BE
S123EDC018085A26F5CEEDF8DFE08603973C4F5FDD38DD3ADE618680A7228D1FCEEE35DF68
S123EDE0EFCEEE3BDFCBDFCE4F5FDD3DDD3FDD41FEFFCCAD007EE0038D013BDE61EC16F3FC
S123EE00FFCAED168680A7237A003C26278602973CDC38C30001DD38DC3A27181A933826A7
S123EE201318DE3D31317C0019DC29DD45DC2BDD477EF4423918DE3F26EC3BDE618630A734
S123EE402518DE4126E03BBDE3BA810D2604CC000039CEEE70BDE39C250E08A60026FB0888
S123EE6008086D0026EF20E6EE01AD00CC0001394C49535400EEC452554E00F1584E45573E
S123EE8000F2C4434F4E5400F2AF434C45415200F2D8455341564500F2EF454C4F414400F8
S123EEA0F3534C4C49535400F38D4155544F535400F3984E4F4155544F00F3A34652454507
S123EEC000F3D400BDE10EDC041A9306260139BDE05BBDE3BABDE1BB2427BDE16CDD12BD1C
S123EEE0E3BA812D270ADC12DD141A930C232139BDE3C3BDE16C1A930C2302DC0CDD142039
S123EF000F810D270139DE04EC00DD12DC0CDD14DC121A9314230139DC12BDEBE6DF6ADCAC
S123EF2014BDEBE6EC001A93142603E6023ADF14DC6A1A9314260139DE6AEC00080808DFAE
S123EF406ABDEB17DE6AA600817D270D4D2B05BDEFD720F0BDEF6320EBBDE110DE6A08DF5D
S123EF606A20CDDE6AA60084EFCEEF81A100270C0808086D0026F586087EEA95EE01AD00FC
S123EF803984EF8EA2EFC3A8EFCAA4EFBC00DE6A08EC00D3080808DF6A8FA601BDFEB8A670
S123EFA0022703BDFEB839DC6AC300068FE60008A600BDFEB8085A26F7DF6A39DC6AC300C6
S123EFC00320E9DC6AC3000120E2DE6A08EC000808DF6ABDEB1739DE6AA60008DF6A817F49
S123EFE026037EF01B810A26037EF033810C26037EF02B8136260CDE6AA60008DF6ACEF1D0
S123F0000A2003CEF04CA100270C0808086D0026F586087EEA95EE017EE11CDE6AE6000816
S123F020DF6A8620BDFEB85A26FA39CEE246BDE11C2006CEE2EABDE11CDE6A08A600810D09
S123F040260408DF6A39BDFEB80820F001E24E0DE2550EE25D0FE26812E27113E29614E26C
S123F0609C15E2A638E96339E96816E2AC03E2B504E2C305E2CA17E2D218E2E306E2F10725
S123F080E2F919E3021AE2DA3AE9C337E9C07CF1487BF1467AF14402F14308E30B79E54413
S123F0A010F14A11F14C20E51D21E52422E52A30E53E31E54132E53233E53634E54435E57E
S123F0C03A40E50A41E50D50E51051E51352E51671E54E60E51972E5487EF14E09E3131B3D
S123F0E0E31A1CE3211DE32A1EE3331FE33C78F15623E34524E34F25E27926E28327E35787
S123F1000BE35F28E28C29E3670001E78502E78D03E7B104E79505E79C06E7A307E7AA08DF
S123F120E7B809E7C00AE31A0BE7D70CE3210DE32A0EE3330FE33C10F15011E34F12E7CFD4
S123F14013E35F003A003B002C00280029002000504F525445002300BDE10EBDF283860132
S123F160971D18DE04189C0626013918EC00DD297D001B2712865BBDFEB8DC29BDEB17864A
S123F1805DBDFEB8BDE110183C18E602183A18DF2B1838C603183A8D3018E60018088D2929
S123F1A05A58CEF1D93AEE00AD007A001A2603BDF25C8D1518A600817D260A1808189C06FC
S123F1C026A97EF4C5180820CE18A6002B0A817E270425041808180839F3E9F3E9F611F7A2
S123F1E07AF7D1F5FCF601F5B6F709F3E3FA37F3E3F8F1F914F47600000000F433F553F496
S123F200A2F94EF811F4B5F4C5F4E9F52EF977F5D6F5F0F5F4F5F8000000000000FA1AFA92
S123F2202CFA4CFA63FA81FAA3F605BDE10E18DE4B18EC00DD29C603183A8D8D18E60018A6
S123F240088D865A58CEF1D93AEE00AD00BDF1C918A600817D260139180820DE860A971A7E
S123F2609D9E2601399DA1810327013918DF31BDE110CEEB06BDE11CDC29BDEB17BDE1100B
S123F2807EE016BDF2D8DE53DF1FDE4FDF21DE57DF23DE5BDF25DE5FDF27DE0A08DF2D7FE1
S123F2A0001E860A971A7F001CCE0000DF3339BDE10E7D001C260618DE317EF1B28625973C
S123F2C0187EEAD3FEFFC4A60A8155260786FFA70ABDFA11BDECF739BDF286DE08A60027A4
S123F2E008080808BDE64F20F4DE0A08DF2D39DC041A9306260139DC0A93041AB3FFC6238A
S123F3000586377EEA95FEFFC418CE0004C604D71A18EC00B3FFC0A700BDFA110817A70019
S123F320BDFA1108180818087A001A26E418EC00A700BDFA110817A700BDFA11FEFFC41841
S123F340DE0418A600A70BBDFA11081808189C0A23F039FEFFC418CE0004C604D71AEC000B
S123F360F3FFC018ED000808180818087A001A26EDEC0018ED00FEFFC418DE04A60B18A7BF
S123F38000081808189C0A23F318DF2D3986019737BDEEC47F0037398655FEFFC4A70ABD53
S123F3A0FA113986FF20F3FEFFC4FCFFC4C3000BDD04FCFFC4E302C3000BDD06EC06A30450
S123F3C0F3FFC0DD0AFCFFC0DD08188FFCFFC4E3048F20A8BDE10EDC10932DBDEB17BDE197
S123F3E010393918E600183A3918A6008D0E37361808BDFAFDBDFBA438ED003918A6008567
S123F40002261D8510260F18EC01D308C3000337C603183A3339BDFB7B3C3005E30038397D
S123F420851027E3BDFB7B3C37363005E30031313020E97D00192704DC06DD2BDE2B9C0644
S123F4402604DE042007EC00CDA30122F5EC00CDA30127102505861B7EEAECE6023A9C068A
S123F46027F420E98F188F7D001927067F00197EF1BD313120F9183C7D0019270718DE0618
S123F48018092004C603183ABDF1C9DE2709099C5D2405861C7EEAECDF271AEF0018387E85
S123F4A0F433DE279C5F2605861D7EEAEC1AEE000808DF2739CEF4D4BDE11CDC29BDEB1794
S123F4C018DF312007BDE1108601971CCC0000DD297EE0160A0D53544F50504544204154C0
S123F4E0204C494E4520232000DE2509099C592405861E7EEAECDF251AEF00C6013718DE31
S123F5002B260139183C189C0627BADE2BE6023ADF2BC603183ABDF1C918A60018383381E4
S123F5201926015C811A26D55A26D27EF472DE259C5B2605861F7EEAEC183C1AEE00BDFA2E
S123F540FDBDFBA4260A1838DE250808DF252002313139BDFAFDBDF1C918A600361808BDFE
S123F560F1C9DE1FEC002A07260586207EEAECEC008300012717ED00C603183ABDF1C91849
S123F580A600817D27E41808BDF1C920E2BDFBA432811226037EF433183CC603183ABDF113
S123F5A0C918A600817D270B817A27071808BDF1C920E77EF4881808BDF1C9BDFAFDBDF1D6
S123F5C0C91808BDF1C9BDFAFD1808BDFBA48FBDFBA48FE70039C600DE613A3C1808BDFAAB
S123F5E0FDBDFBA44D2705862E7EEAEC38E70039C60420E4C60320E0C60820DC86FF971B3D
S123F600397F001B390F07847F06CF078A80060E39BDF84F18A600817D2704817A2607BDBE
S123F620E1107F00373981A22616183CC60218EB01183A3808E600C0020808BDF8CD203942
S123F6408136261E18A60181072605BDF6B6202981022605BDF6CB2020810B2605BDF6DFD2
S123F660201781122605BDF6D7200EBDFAFDBDFBA4BDEB178620BDFEB8BDF1C918A600813B
S123F6807C2708817B2628180820131808D61EC40750CB0827088620BDFEB85A26FABDF1AC
S123F6A0C918A600817D270A817A27067EF626BDE1107F0037398D432705862A7EEAECD160
S123F6C01E23078620BDFEB820F5398D2E2704862B20E9177EFEB88D222708863220DD8D6C
S123F6E01A8D0117368D0332200444444444840F8B30813923028B077EFEB8C603183ABD50
S123F700FAFD1808BDFBA44D3918A6008510260586217EEAEC18EC01D3088FEC0327048664
S123F7202220EF3CC604183ABDFAFD180838DC2DED03C30002DD2DBDFBA42A0486272018F9
S123F7403CEE03ED00C300013805D32D1A932D23051A9310230586097EEAECDD2DEE0308BD
S123F760086F00089C2D26F9BDF1C918A600817D27071808BDF1C9209039DC2383000A1A97
S123F7809355240586237EEAECDD23183CBDF3FC1838DE23ED00DC29ED08BDF3E9BDF1C90F
S123F7A01808BDF1C9BDFAFDBDFBA4DE23ED04CC0001ED02BDF1C918A600813A27041AEFCC
S123F7C006391808BDF1C9BDFAFDBDFBA4DE2320E1BDF3FCDE231AA300270586247EEAECA9
S123F7E0183C1AEE0018EC00E30218ED006D022B111AA3042F1118388FC3000ADD23BDF1B5
S123F800C9391AA3042DEF18381AEE06EC08DD29398D3C18A60081A2261B183CC60218EB6A
S123F82001183A3808E600C0020808BDF8CD1808BDF1C92003BDE110CEF84CBDE11CBDE026
S123F840BB8D3B25F0BDE1107F0037393F200018A60081782701391808BDF1C9BDFAFDBDF0
S123F860FBA42A0586307EEAEC1A83000722F5D737BDF1C9817D27051808BDF1C939BDE0D5
S123F8805B810D26020D398D17BDF1C918A600817D270B817A27071808BDF1C920E00C39FF
S123F8A081242608BDE3C3BDE6CC2003BDF8DA3736BDE05B812C2709810D270886157EEAEB
S123F8C0ECBDE3C3BDF3FC8F3233ED00395D2709A60008BDFEB85A26F739BDE3BA812D2683
S123F8E00CBDE3C3BDE69E4353C3000139BDE69E39DE3326048D1DDE33DF00BDF87E250515
S123F900DE00DF3339183C18DE00180818088D3A183820DD183C18DE04183C18E602183A28
S123F92018DF331838C603183ABDF1C918A600810C270D18DE33189C0626DE86267EEAEC51
S123F9401808180818DF33183839183C20E8BDFAFDBDF1C91808BDF1C9BDFBA427037EF49A
S123F96033C603183ABDF1C918A600813926071808BDF1C920E8391808BDF1C9BDFAFD18DE
S123F980081808BDFAFD183C18DE1F18EC022B061A8300FF230586287EEAEC05C3B6008F14
S123F9A0A60081FF27028D1D08A60081FF27028D1418A6018D320918A6008D2C1838BDFB4C
S123F9C0A4BDFBA439183C18DE61C61618E73BA70007360FC61718E73B8D36C61618E73B46
S123F9E03206186F3B183839183C18DE61C60218E73BA7003607360FC60318E73B8D12C642
S123FA000218E73B3206186F3B32A10026DF1838393CCE0D020926FD3839BDF84FBDF3FCE5
S123FA208FBDFED5164FED007F0037391808BDFAFDBDFBA4DD38391808BDFAFDBDFBA44D67
S123FA40270586357EEAECDE61E727398D4ABDFAFDBDFBA4DD3ABDF1C91808BDF1C918DFDE
S123FA603D20198D33BDFAFDBDF1C91808BDF1C9BDFBA42604DD3F200318DF3FC603183A74
S123FA80398D15078510260586347EEAECDC45DD29DC47DD2B31313B7D0019270586337ECA
S123FAA0EAEC398DF3BDFAFDBDF1C91808BDF1C9BDFAFDBDF1C91808BDF1C907360F18DFEC
S123FAC041BDFBA41A830001230586367EEAEC86105D270148DE61A724BDFBA42608DE6179
S123FAE06F26DD4120101A83000422DECB0358585858DE61E7263206C603183A398610BD25
S123FB00FC0618A6008110260818088DF0180820F14D2A048D1220EABDFBB3BDFBF6240132
S123FB20391808BDFC0620DA8184260E18EC01D3088FC603183AEC03202D81A4260DCDEE9D
S123FB4001C60418EB03183A8F201C819426138D2A183C3C05183018E3003818388FEC00D3
S123FB60200586087EEAECDE1F09099C512407861797187EEAECDF1FED003918EC01D308AF
S123FB808FEE03260586187EEAECC604183A3CBDFAFD180838BDFBA41AA300230486192061
S123FBA0E60808393CDE1FEC000808DF1F381A83000039813627013918A6014AC603183A95
S123FBC01658CEFBD03AEE00AD00180818A60039FE0BFE89FE30FDB3FE61FDC4FE89FDD646
S123FBE0FDE1FDF0FE89FE99FEA8FEACFEB0FEB4FE8EFE89FE9281112708817A24020C399E
S123FC0086118D020D39DE21099C4D260586177EEAECDF21A700DE21A60081102719E60163
S123FC20C4F084F0112210A601E600C1112609811026050808DF2139E70108DF218D022023
S123FC40D5817025078070CEFC8F203C816025078060CEFC952031815025078050CEFC973E
S123FC602026814025078040CEFC9D201B813025078030CEFCA12010812025078020CEFC8C
S123FC80AD200586087EEAEC16583AEE006E00FD6BFD6CFD75FDB2FD3DFCEBFD37FCD5FC94
S123FCA0DEFD7DFD88FD8EFD94FD9AFDA0FCCAFCBFFCB3BDFBA4DE1FA800E801ED0039BD16
S123FCC0FBA4DE1FAA00EA0120F2BDFBA4DE1FA400E40120E7BDFBA4DE1FE30020DEDE1FBD
S123FCE0EC02A3000808ED00DF1F398D08BDFBA4DE1FED0039DE1FA600A80236EC0026058D
S123FD00861A7EEAEC2A03BDFD756D022A09EC024353C30001ED02EC00EE028F023CDE1F10
S123FD20ED023233ED00324D2A0CBDFD75EC024353C30001ED02398DBCBDFBA439183CDE1A
S123FD401FA601E6033D37361830A601E6023D18EB0018E700A600E6033D18EB0018E70062
S123FD6008083233ED00DF1F18383939DE1FEC004353ED00398DF5C30001ED00398D272C6C
S123FD80026C030808DF1F398D1C2FF720F38D162EF120ED8D102DEB20E78D0A26E520E197
S123FDA08D0427DF20DBDE1FEC026F026F031AA3003939BDFAFDDE1FEC002A054353C3008B
S123FDC001ED0039BDFAFDDE1FEC0027F4CC00016D002AED20E6BDFAFDDE1FEE00AD00207D
S123FDE00ABDFAFDDE1FEE00E6004FDE1FED0039BDFAFDDE1FEC001A8300FF230586287E71
S123FE00EAEC05C3B6008FEC0020E0BDFAFDBDF1C91808BDF1C9BDFAFDDE1FEC02EE0003BD
S123FE202804862C20D98FDE1F0808ED00DF1F39BDFAFDDE1FEC002B061A83000723048608
S123FE402D20E1DE61E7306D302AFC4FE631EB328900EB338900EB3489000404DE1FED000A
S123FE6039BDFAFDDE1FEC00270C2B04DC352015DE61EC0EDD35DC35581BD6360505D33513
S123FE80C33619DD3504ED003986297EEAECDC38200FDE61E6274F2008C600DE613AE600E2
S123FEA04F180918097EFB67C60420EFC60320EBC60820E7C60A20E37C001E373CCE00B4E9
S11FFEC0D637583AEE0026087F003786317EEAECAD00383339373CCE00A420E46C
S123FF008D0D36B69800850227F932B7980139B69800850127F9B698013936B698008501D7
S123FF2032393CDE61A62E842027FAA62F38393CDE6136A62E858027FA32A72F38393CDEBA
S123FF406136A62E85203238398D2A8D11867E979E97A1CCFF1ADD9FCCFF0FDDA2393CDE17
S123FF60618630A72B6F2C860CA72D861197438613974438398613B798008656B7980039F1
S117FF808DBC270E368D9B914426068D95914326FA32209B89
S123FFA0FF00FF22000000000000000000000000FF02FF800000000000000000000000009D
S113FFC0C0002000600020001000F424FF4940001D
S123FFD600C400C700CA00CD00D000D300D600D900DC00DF00E200E500E800EB00EE00F15F
S10DFFF600F400F700FA00FDED71BD
S903E00319
